:03000000021B4898
:0C1B480078FFE4F6D8FD7581D502003668
:0100190022C4
:061853008B318A3289335B
:101859007571027F481219BC121B94EF20E0F9AB95
:1018690031AA32A9331205377879E6FE08E6FDED8B
:01187900FF6F
:01187A00224B
:100F500043525354005341564500434647002D3EEB
:100F600053320052415445434C5220554E4954424D
:100F70004C4E4B5452494754524556535452545375
:100F8000544F505A45524F44464C54534156455283
:100F9000535420535720202E3235203173202032D5
:100FA000732020357320203130732033307320318B
:100FB0006D2020326D2020356D202031306D2033A2
:100FC000306D2031682020326820203468202000D5
:100FD0000000010004000800140028007800F0015F
:100FE000E004B009601C2038407080E1004665656F
:100FF00074596172644D6574724F6666204F6E203D
:10100000204E6F2020596573204F66662054696D0D
:1010100065416C7420547269674F66662054696D2F
:1010200065416C74204F6666205472696750777210
:05103000205265632061
:10187B0025E024CFF582E4340FF583220533E533DD
:10188B00C394022208F608F608F62275F004A42485
:05189B00F9F9740F22B1
:1013FD00789976AB0876CD087600087604E408F681
:10140D0008760108F60876FA08764012188F08F665
:10141D0078A7F608760A08F608763C08F6087614DA
:10142D0008F608760F12188F7BFF7A0F7950121776
:09143D009A7F051216C70217FD83
:1019D70075751D7576C01216FD789AE664CD70048C
:0919E70018E664AB60031213FD65
:0119F00022D4
:0D1B1000C2AF7DC07C1DE4FF121A7AD2AF77
:011B1D0022A5
:1016FD00753EFF85753F85764075410075420075D5
:10170D004399E4FFAB3EAA3FA9408F827583001237
:10171D00050AAB41AA42A9438F8275830012054980
:04172D000FBF1AE0F0
:011731002295
:1017FD007D01E4FF1219467BFF7A0F795512179A76
:10180D00121B10C2AF7F997B1A7DC07C1D121A84EA
:0D181D00D2AF7F021216C7E4FDFF0219468C
:10073500E4F5317BFF7A0F795A12179A7F05121665
:10074500C7A297829650FAA2969217A2979218E599
:100755003175F004A42463F9740F35F0FA7BFF12A8
:10076500179A7F051216C7853132E4F5337BFF7A78
:100775000F795E12179AE531B40900507790078911
:10078500F82828730207A40207F90207C50207CD56
:100795000207D10207D90207E10207E90207F17F43
:1007A50001EF12187B789BE6FC08E6FD7401936D5A
:1007B5007003E4936C70028F330FBF0FE402087C63
:1007C500789DE6F5330208A2789E800278A6E6F5C4
:1007D500330208BC78A5E6F5330208E378AFE6F501
:1007E5003302090078B0E6F53302091D78B1E6F564
:1007F5003302093AE53165326003020754A2173026
:100805009601B35013A296921730960C0531E53137
:10081500C3940C4003E4F531A218309701B350D4CA
:10082500A29792183097CDE531B40C0050C69008C8
:100835003AF828287302085E02088A02089002081E
:10084500AE0208C20208D50208EE02090B02092809
:1008550002094E02095402095A0533E533C3940FC0
:100865004003753301E53312187BE493FF7401935C
:10087500789BCFF608EFF6E53375F004A42493F9D9
:10088500740F0209431213090207F90533E533C34F
:1008950094034003E4F533789DA633E53375F004FE
:1008A500A424EDF9740F0209431218874003E4F5F7
:1008B50033789EA633E5331218960209431218873A
:1008C5004003E4F53378A6A633E533121896806E17
:1008D5001218874003E4F53378A5A633E53375F0A0
:1008E50004A42401F9741080550533E533C3940439
:1008F5004003E4F53378AFA633E53375F004A4245B
:1009050009F9741080380533E533C394034003E4D3
:10091500F53378B0A633E53375F004A42419F974DA
:1009250010801B0533E533C394044003E4F53378A5
:10093500B1A633E53375F004A42425F9741035F018
:10094500FA7BFF12179A0207F91213FD0207F91233
:0B09550017FD0207F943A2080207F992
:0A1B60004552415300444F4E45002A
:10198200E4D3FCFD7B80FAF9F8020696789BE6F533
:0D1992005508E6F55622E56AAE6978062292
:1011EA00C215C216E4F532F533AE32AF33121982A4
:1011FA00401CE53164816016AF33AE321217CC124F
:10120A001A668F310533E53370DF053280DBE5314D
:10121A00B48108E533153370021532AE32AF33E4C8
:10122A00C3121984700CD215121B2CE4F569F56AE5
:10123A00800785326985336AE4F56BF56C755480ED
:03124A0012198EE8
:01124D00227E
:0417CC008F828E83F7
:1017D0001219824027E582AE837806C333CE33CE1A
:1017E000D8F9FD757102EE7879F6CFEDCFEF08F6F6
:0C17F0007F50121A24121B94EF20E0F925
:0117FC0022CA
:0319F100CDEFCD6A
:1019F400757102EE7879F6ED08F67F50121A24120A
:061A04001B94EF20E0F945
:011A0A0022B9
:101A66007571017F501219BC121B94EF20E0F978B2
:031A760079E6FF0F
:011A7900224A
:101A51001219F1E4FFFE0FBF00010EBE0FF8BFA087
:041A6100F5121A66FA
:011A6500225E
:06173200CBEFCBCAEECAAA
:10173800301503301627757103EA7879F6EB08F649
:1017480008EDF67F50121A24121B94EF20E0F9E4FA
:0D175800FFFE0FBF00010EBE0FF8BFA0F591
:011765002261
:10155600753400753500753654E4F533121998C3A1
:1015660033CE33CED8F97C002533FFEC3EFEAB34C8
:10157600AA35A93685338275830012050AFD12172E
:10158600320533E533C3940640D2756B00756C069D
:011596002232
:1010FB008E318F32121998C333CE33CED8F9256C7B
:10110B00FFE56B3EFEEEC0E0EFC0E0E531FDD0E069
:10111B00FFD0E0FE121732056CE56C7002056B1206
:10112B001998C333CE33CED8F9256CFFE56B3EFE51
:10113B00AD32121732056CE56C7002056B0558E584
:10114B005870020557C3E56C9440E56B940040174B
:10115B00E4F56BF56C056AE56A70020569AE69FF2B
:08116B001219825002D2152274
:10130900E4F56BF56C7BFF7A1B796012179AD2169C
:10131900E4F53EF53FAE3EAF3F1219824021E53F6D
:10132900AE3E7806C333CE33CED8F9F56C8E6B7DDD
:1013390081FF121732053FE53F70DA053E80D6C2BC
:10134900167BFF7A1B796512179AE4F569F56AF538
:051359006BF56CC215EC
:01135E00226C
:1012B200E4F53EF53FF540F541AE40AF41121982EB
:1012C2004044E53F6481603EAF41AE401217CC120C
:1012D2001A668F3FE53F64807022AF3E053EFCFDFB
:1012E200FEFBFAF9120D277F2C120016AE40AF4119
:1012F200E4FCFDFBFAF9120D27121B7D0541E541C5
:0613020070B7054080B346
:0113080022C2
:021446008F3ED7
:10144800E4F53FF540F541F542AE41AF421219824D
:101458004030E5406481602AAF42AE411217CC1299
:101468001A668F40E540B4800FE53F653E7007AFD0
:1014780042AE410217CC053F0542E54270CB05411B
:0214880080C71B
:01148A00223F
:1015970012198E78A6E6F559E4F557F5581215563F
:1015A70085696D856A6E7F0112124E30021A78A91D
:1015B700E6FE08E6FFE4FCFD7B64FAF9F812056B2A
:1015C7008F668E658D648C63300505C205121A3BE4
:0115D70022F1
:10168F00856931856A32E56C456B60080532E53254
:10169F0070020531856D69856E6A1215568531693F
:1016AF0085326AAE31AF321219825007E4F569F50F
:0816BF006AD2157F0202124EEF
:101A7A00740478FF769612FF0322740078FF769634
:041A8A0012FF032222
:0300330002103583
:0D103500C0E0C0F0C083C082C0D075D008FC
:10104200E5D954F8FF12070F106F08106F10107EC9
:1010520018109920108028109930109B3810A14048
:1010620010994810BA5010D758000010E58574DA6C
:10107200C2DDC2DC7572007573008070800EE5718E
:10108200700280560573E573700205721200268F96
:10109200DAC2DDC2DC80558016D2DDC2DC804DC2F0
:1010A200DDC2DCE5717004C2DA8041D2DA803DC271
:1010B200DDD2DC756F048034AFDA121B540573E5A0
:1010C2007370020572C2DDC2DCE5717004C2DA809F
:1010D2001BD2DA8017AFDA121B54C2DDD2DC756F75
:0E10E200028009756F04C2DDC2DCD2DAC2DB07
:0B10F000D0D0D082D083D0F0D0E0320E
:10182A0043910C43920CE4F5DBEF25E0F5DB30172E
:10183A000343DB0175DD2575DC2575D84453F8FEB5
:09184A0053F7FEE4F56FD2E82229
:101A2400E56F30E002FF22E4F570756F03EF25E007
:071A3400F574D2DD7F0222F0
:1019BC00E56F30E002FF22E4F5701571756F05EFED
:0B19CC0025E04401F574D2DD7F02220B
:061B940020DBFDAF6F2213
:0D0026001571AF70057074792FF8E6FF2298
:0C1B540074792570F8EFF6057015712209
:0E1B1E00E4F5847585FFF592F5A475A5FF2208
:071B8600EE3395E0FDFC22A7
:1018A000C212C214C211D2A2C2A0C2A1E4FDFF1290
:1018B0001946E4FD7F011219467F0812124E7F047B
:0318C00002124EC3
:10194600EF146011047016BD0104C2A78002D2A76D
:0E195600A2A7921322BD0103C2A622D2A6228E
:10124E00EF14B40800505C90126375F003A4C583CC
:10125E0025F0C5837302127B0212810212880212DC
:10126E00940212960212940212A00212A8D21275C1
:10127E00190122C212A21392A722D214751A057D49
:10128E00017F010219468005C211C28722C211D206
:10129E008722D211D28775180122C2A47F0112169D
:0412AE00C7D2A422DD
:10161700301212D5190F30A707C2A775191E8005FA
:10162700D2A7751946E51AD39400400CD51A09C2FA
:1016370014E4FD7F01121946301111D5180E3087B9
:0D16470006C28775180522D28775181E226D
:10190600C374039FFE1392A0EEA2E192A1AF80CF13
:0F1916005480CFED547FCF4FCF8F80C2A2D2A28B
:01192500229F
:06179A008B408A418942E8
:1017A000E4FCCFECCF7D201219060CBC04F4E4FC61
:1017B000AB40AA41A9428C8275830012050AFD60E4
:0B17C0000ACFECCF1219060CBC04E5A8
:0117CB0022FB
:041173008F828E8356
:10117700121B86E47B0F7A27F9F8C31206965003F1
:1011870090270FAF82AE83121B867B197AFC79FFFB
:1011970078FFD3120696400390FC19E4F531741BCF
:1011A7002531F8E4F60531E531B405F2AE83AF82B7
:1011B700121B867B007A00791B120D27E51E701A19
:1011C700753103741A2531F8E6FF741B2531F8C60B
:1011D700EFC6D531EE751B2080E27B007A00791BC4
:0311E70002179A52
:1019640046554C4C0050524F47005A4C4F47004D7F
:0E1974004F44310076322E3100547269670004
:101ACA00E6FE08E6FFE4FCFD2278CE1206D178C6CF
:031ADA000206EA17
:030013000218E5EB
:1018E500C0E0C0D075D010200E0CAF8DEFAD8BF5DC
:1018F5005EEDF55FD20E758D00758B00D0D0D0E012
:0119050032AF
:0216C7008F3F53
:1016C900E4F540F541C3E541953FE54094005023D9
:1016D900900000AF82AE83E4FCFD7B207A4EF9F8DE
:1016E900D31206964003A380EA0541E54170D60569
:0316F9004080D25C
:0116FC0022CB
:0E1B2C007BFF7A19796412179A7F0A0216C796
:0F1B0100D20B301506121B2CC20B221215972285
:05000E00C20B02168F79
:101A3B0078D21206F600000000121AD378CE1206E6
:061A4B00F600000000227D
:10003600121B1E121B6A1218A07F041216C72097E5
:10004600127BFF7A19796912179A7F0112148BD2E3
:10005600AF80FE2096091204E41211EA1207357ADF
:1000660019796E1204D97A1979731204D97BFF7A39
:1000760019797812179A7F041216C7E4FF12148BA7
:100086001204E47F011216C71211EA120019C21AED
:100096001216547F011216C7E4F560F56112001AB4
:1000A600A2969208A2979209E4F52478CA1206F657
:1000B60000000000E4F52578D21206F6FFFFD8F11D
:1000C60078C61206F600000000E4F55378CE120654
:1000D600F600000000C20DC20BC20CE4F567F5681D
:1000E600F526F527F55EF55FC20EF562C20FF55DE2
:1000F600F55CF55BF55AF566F565F564F563F5208F
:1001060078AFE624FE600B14600C2402700AD2015C
:100116008006D2068002D20078B0E624FE6007048C
:100126007006D2028002D20778B1E624FE600B1474
:10013600600C2402700AD2038006D2048002D20523
:10014600300117C20178A7121ACA7B64FAF9F812AD
:10015600056B8F5D8E5C8D5B8C5A301AFDC21A3032
:100166000C33A208309601B3400BA209309701B3B5
:10017600400302024730961230970FC20CE4F5672F
:10018600F5687F0412124EE4F553A2969208A297E0
:100196009209020247209605209702D21030965601
:1001A600309753301031C21078C61206D1EC4D4E3E
:1001B6004F78D2700C1206F600000000121AD38097
:1001C600101206F60000000078C61206F6000000BF
:1001D60000D209D2088024789EE6601F0568E5688B
:1001E60070020567D394B8E567940B400ED20C7F76
:1001F6000512124E8005E4F567F568A208309601EF
:10020600B3501FA2969208309618201015C201E529
:10021600536007E4F5537F0680057553017F071287
:10022600124EA209309701B35017A2979209309740
:100236001020100DB20B300B05121B0180031200AB
:100246000E120960AF5DAE5CAD5BAC5AEC4D4E4F25
:10025600602674FF2FF55DEE34FFF55CED34FFF597
:100266005BEC34FFF55AAF5DAE5CAD5BFC4D4E4FBB
:100276007006200B03121B01AF66AE65AD64AC635E
:10028600EC4D4E4F602374FF2FF566EE34FFF56597
:10029600ED34FFF564EC34FFF563AF66AE65AD642F
:1002A600FC4D4E4F700312000E200E03020357C280
:1002B600AFC20ED2AFE4855F30855E2FF52EF52DE9
:1002C600AF30AE2FAD2EAC2D7B107A27F9F8120584
:1002D6006B8F308E2F8D2E8C2DE4FB7A90F9F812D1
:1002E60014CF8F308E2F8D2E8C2D78A5E66009C306
:1002F60074B89FFF740B9EFEE56214601624FE60C0
:100306002024037049C3EF94B0EE9404500E756236
:10031600018009D3EF9414EE94054035756203808D
:1003260030C3EF94B0EE9404502775620130000696
:10033600200B03121B01300305C203121A3B300BBC
:1003460002D20F7BFF7A19797D12179A8003E4F5A2
:10035600620525E525C3940550030204D3E4F5257B
:10036600FB7A0079281218538E298F2AE528640211
:1003760060030204D378CA1206DDE8C0E0E9C0E0F3
:10038600EAC0E0EBC0E0789DE6FDAF2AAE29121385
:10039600B1D0E0FBD0E0FAD0E0F9D0E0F8EB2FFFE7
:1003A600EA3EFEE93DFDE83CFC78CA1206EA052471
:1003B600E524C3940550030204D378CA1206D1E497
:1003C6007B05FAF9F81214CF78CA1206EA78CA122F
:1003D60006D178C61206DDC3EF9BFFEE9AFEED99B5
:1003E600FDEC98FC78CA1206EA78D21206D178CAD1
:1003F6001206DDD3120696400A78CA1206D178D2C2
:100406001206EAE553600A78D4E6FE08E68E2BF576
:100416002C78CCE6FE08E68E29F52AE5536006AF71
:100426002CAE2B8004AF2AAE29121173300B4E0569
:1004360027E52770020526C3789C96E52618964080
:100446003CE4F526F5277F0312124E300D0DE52903
:10045600FF120016AF2AE52A12001620151A78A6F2
:10046600E6600C300F097F007E821210FBC20FAFD0
:100476002AAE291210FB8005121B2CC20B78CA1259
:1004860006D178CE1206EA78CA1206F600000000F7
:10049600E4F524300405C204121A3B30061678AB84
:1004A600121ACA78CE1206DDD31206964006200B23
:1004B60003121B0130071678AD121ACA78CE12063F
:1004C600DDC31206965006300B0312000E121617E5
:0304D600020160C0
:1004D9007BFF12179A7F041216C722D2AF1219D7BF
:0804E900C2177F7012182A22CD
:1018C300444C0021536967005A4C4F47004D4F4425
:1018D3003100322E31004D617920323520323030E3
:0218E3003400CF
:10151300AF39AE38AD37AC36EC4D4E4F22EF24FF2A
:10152300F539EE34FFF538ED34FFF537EC34FFF5DC
:101533003622E475392075384EF537F53622E475D1
:101543003901F538F537F5362275330075340075F2
:03155300359922A5
:10096000121B3AEF7003020B5D7F0412124EE4F586
:1009700053C20CF567F56812199FEF12070F0B5160
:10098000240B5A2A0AAF5209A3610A31630A846C04
:100990000A8A720A87730AB3740B26760B1E7800D4
:1009A000000B5D7BFF7A1879C312179A1215351266
:1009B0001B3AEF700A121513600512152080F01211
:1009C00015137003020B5D12199F8F32121446E447
:1009D000F539121545E47F06FEFDFCAB39AA38A9AE
:1009E00037A836C31206AC501F121A668F32120097
:1009F00016E5392401F539E43538F538E43537F5AD
:100A000037E43536F53680CD121A668F32E532641A
:100A1000806016E53264816010120016121A668F2B
:100A2000321200167531018003E4F531E53170D8DA
:100A30002212154C121541F53212151360241215AD
:100A400035121B3AEF700A1215136005121520803B
:100A5000F01215136003120B5E0532E532C3941ACF
:100A600040D7121513601A7899B6AB0708B6CD03B4
:100A7000020B577BFF7A1879C612179A7F0A021663
:100A8000C7020B1BB20D220212B212154CE4F53252
:100A9000AB330535E535AA347002053414F9120478
:100AA000F1FF1200160532E532C3941A40E22243E8
:100AB000A20822753300753400753577121541F59B
:100AC000321215136024121535121B3AEF700A12F8
:100AD0001513600512152080F01215136003120B18
:100AE0005E0532E532C3940240D7121513602CAE76
:100AF00077AF78EE3395E0FDFC78CE1206DDC3EFDC
:100B00009BF53DEE9AF53CED99F53BEC98F53AAF47
:100B10003D78A3E53CF608EFF6803C0216FD7F0425
:100B200012124E0213097A1879CB120B727A1879C5
:100B3000D0120B727F761200167BFF7A1879D512CD
:100B40001ADD121B7D7BFF7A1879D9121ADD021B80
:0D0B50007DE478A3F608F60217FD1213FDF0
:100B5D002212199FAB33AA34A935853282758300D1
:0E0B6D00EF120549227BFF121ADD121B7D22BA
:0A1B6A00E4F5955396BF53A27F22C5
:101654005389F0438901538FFE758C70E4F58A53E6
:10166400B8FD53B7FDD2A9D28C53890F4389905347
:101674008FEFF58DF58B4391105392EF53B8F753D9
:0B168400B7F7D2ABD28ED28AD2AA22D6
:03000B00021B7461
:091B7400D21A758C70758A0032DA
:03001B00021B8D38
:071B8D00758D00758B00321D
:101A8E000D0A00303132333435363738394142435E
:041A9E004445460075
:101AA200AF52AB46AA47A948055222AF45AE44AD54
:041AB20043AC4222DD
:10148B005387BF75985053877FE4F5BABF01054367
:10149B00A240800353A2BFE4F5BD75BE30F5BF7506
:1014AB00BD035391FE4392014391025392FDC21B24
:1014BB0053B8EF53B7EF43B81078C4F618F678C5A6
:0414CB00F6D2AC2287
:030023000217665B
:10176600C0E0C0D075D01030981E78C4E6C3940F80
:10177600501418E60624B3F8A69978C40618E6C3EA
:10178600941040027600C298309904C299C21BD0C8
:04179600D0D0E0329D
:08000300201BFDD21B8F992286
:1019260078C4E6D39400401508E60624B3F8E6FF2B
:0F19360078C41608E6C394104005E4F6227F003B
:01194500227F
:03001600020003E2
:10199F007F207E4E78C4E67010D3EF9400EE940053
:0C19AF004007EF1F70EE1E80EB1219269F
:0119BB002209
:101ADD001204F1FF600C120016740129F9E43AFAB0
:031AED0080EE2266
:0E1B3A0078C4E6D3940040037F01227F00228E
:101A0B00CEEFCEEE54F0C4540F901A9193FF120008
:091A1B0016EE540F93FF020016B1
:101AF000CDEFCDCCEECCEEFF121A0BCFEDCF021A0C
:011B00000BD9
:091B7D007BFF7A1A798E021ADD51
:0E0D27008F458E448D438C428B468A47894807
:100D3500E4F552EC4D4E4F7017E94A4B70057F3084
:100D4500020016121AA28F827583007430020E4AB1
:100D5500121AAFEC33502AE5484547454670077FE0
:100D65002D120016800D121AA28F82758300742D24
:100D7500120549121AAD1206888F458E448D438C93
:100D850042755101754C00754BCA754A9A75493BB8
:100D9500E4FFFEFDFCAB4CAA4BA94AA849D31206B9
:100DA500AC5003020E35121AADA8491205F68F5044
:100DB5008E4F8D4E8C4DEC4D4E4F7004E55170238A
:100DC500E5502430FFE548454745467005120016B5
:100DD500800EAE52121AA48E82758300EF12054959
:100DE500E4F551AF4CAE4BAD4AAC49AB50AA4FA957
:100DF5004EA84D12056BC8ECC8C9EDC9CAEECAC3E9
:100E0500E5459FF545E5449AF544E54399F543E500
:100E15004298F542AF4CAE4BAD4AAC49E47B0AFA79
:100E2500F9F81205F68F4C8E4B8D4A8C49020D95BB
:100E3500E547454845466010AB46AA47A94885524F
:080E450082758300E4120549E7
:010E4D002282
:100B7B000134C35001DBBF68028BBB800344B798C1
:100B8B000407B3B004D5AFC805A9ABE00689A7F835
:100B9B000775A410086DA02809719C400A8198580C
:100BAB000B9F94700CCA90880DE98CF90E048CA0E5
:100BBB000EA88AAC0F4D88B80FF786C410A184D04D
:100BCB00115182DC120580E812BB7EF413747D0098
:100BDB0014307B0C14F2791815B877241680753005
:100BEB00174B733C1819714818ED6F5419C46D608D
:100BFB001AA16B6C1B7E69781C6167841D4A65901A
:100C0B001E37639C1F2561A8201A5FB421125DC09B
:100C1B00220D5BCC230E59D8241557E4251F55F014
:100C2B00262F53FC27425208285B501429764E205E
:100C3B002A9B4C2C2BC04A382CEE48442E1E465077
:100C4B002F55445C308F426831D1407433173E804E
:100C5B0034633C8C35B13A98370938A4386636B0D2
:100C6B0039C734BC3B2D32C83C9D30D43E0F2EE0EF
:100C7B003F882CEC41062AF8428D29044418271092
:100C8B0045AB251C4741232848E121344A861F40A8
:100C9B004C311D4C4DE21B584F9C1964515D177024
:100CAB005323157C54EF138856C4119458A20FA0EC
:100CBB005A830DAC5C6D0BB85E6009C4605807D0ED
:100CCB00625A05DC646203E8667301F4688A00000B
:100CDB006AA1FE0C6CB8FC186ECFFA2470E6F830E3
:100CEB0000000000000000000000000000000000F9
:100CFB0000000000000000000000000000000000E9
:100D0B0000000000000000000000000000000000D8
:0C0D1B00000000000000000000000000CC
:1015D80075F004E538A4247BF582E5F0340BF58337
:1015E800E49322FE740193FF75F004E538A422F514
:1015F80083C37401939FFFE4939EFEE4228F398E88
:0F160800388D378C36228F358E348D338C3222CD
:101AB600C3EF9DEE9C400AD3EF9BEE9A50037F0145
:041AC600227F002259
:040E4E008E368F3716
:100E5200E4F5381215D8FC740193FD1215F0247FC5
:100E6200F582E5F0340BF583E493FA740193FBAF5A
:100E720037AE36121AB6EF7003020F3E1215D812B1
:100E820015EB247FF582E5F0340B1215F78F3C8EBB
:100E92003BF53AF5391215F02481F582E5F0340B71
:100EA200F583E4931215EB247DF582E5F0340B1201
:100EB20015F78F408E3FF53EF53DAD3EAC3D120637
:100EC200888F408E3F8D3E8C3DAE36AF37E4FCFDC1
:100ED200EEC0E0EFC0E01215D8FE740193FBCAEE3B
:100EE200CAD0E0FFD0E0FEC3EF9BFFEE9AFEED9486
:100EF20000FDEC9400FCAB40AA3FA93EA83D1205C0
:100F02006BAB3CAA3BA93AA8391214CFC8ECC8C9AA
:100F1200EDC9CAEECACBEFCB1215F0247DF582E5FE
:100F2200F0340BF583E493FE740193FFE4FCFDEBD4
:100F32002FFFEA3EFEED39FDEC38FC220538E5389C
:0D0F4200C3946A5003020E55E4FFFEFDFC4F
:010F4F00227F
:01001A0022C3
:10135F00121605AB39AA38A937A836E8C0E078A12C
:10136F00E6FE08E6FFE4FCFDD0E0F812056B12166E
:10137F0005780E1206BD12160578A3E6FE08E6FFE5
:10138F00EE3395E0FDFCE5392FF539E5383EF538BC
:10139F00E5373DF537E5363CF536AF39AE38AD3785
:0213AF00FC221E
:0213B1008D317C
:1013B300120E4E12160E12135F12160EE531146042
:1013C3001C14702DE47FE87E03FDFCAB35AA34A921
:1013D30033A83212056BE47BE87A0B800CAF35AE91
:1013E30034AD33AC32E47B03FAF9F81214CF12169E
:0913F3000EAF35AE34AD33AC325F
:0113FC0022CE
:1004F100BB010689828A83E0225002E722BBFE0209
:09050100E32289828A83E493223B
:10050A00BB010CE58229F582E5833AF583E02250A6
:10051A0006E92582F8E622BBFE06E92582F8E222F0
:0D052A00E58229F582E5833AF583E493220A
:10053700BB010689828A83F0225002F722BBFE01A3
:02054700F3229D
:10054900F8BB010DE58229F582E5833AF583E8F0E8
:10055900225006E92582C8F622BBFE05E92582C894
:02056900F2227C
:10056B00E88FF0A4CC8BF0A42CFCE98EF0A42CFC2F
:10057B008AF0EDA42CFCEA8EF0A4CDA8F08BF0A4AD
:10058B002DCC3825F0FDE98FF0A42CCD35F0FCEB0C
:10059B008EF0A4FEA9F0EB8FF0A4CFC5F02ECD39D1
:0F05AB00FEE43CFCEAA42DCE35F0FDE43CFC223E
:1005BA0075F008758200EF2FFFEE33FECD33CDCCF8
:1005CA0033CCC58233C5829BED9AEC99E58298407B
:1005DA000CF582EE9BFEED9AFDEC99FC0FD5F0D658
:1005EA00E4CEFBE4CDFAE4CCF9A88222B800C1B982
:1005FA000059BA002DEC8BF084CFCECDFCE5F0CBC0
:10060A00F97818EF2FFFEE33FEED33FDEC33FCEBF8
:10061A0033FB10D703994004EB99FB0FD8E5E4F9B3
:10062A00FA227818EF2FFFEE33FEED33FDEC33FCA0
:10063A00C933C910D7059BE99A4007EC9BFCE99A94
:10064A00F90FD8E0E4C9FAE4CCFB2275F010EF2FD9
:10065A00FFEE33FEED33FDCC33CCC833C810D707D9
:10066A009BEC9AE899400AED9BFDEC9AFCE899F814
:0E067A000FD5F0DAE4CDFBE4CCFAE4C8F922A7
:1014CF00C2D5E830E70FB2D5E4C39BFBE49AFAE448
:1014DF0099F9E498F8EC30E717B2D5121505120513
:1014EF00F6E4C39BFBE49AFAE499F9E498F88003D5
:1014FF001205F630D50DE4C39FFFE49EFEE49DFD7B
:04150F00E49CFC223A
:0E068800C3E49FFFE49EFEE49DFDE49CFC2283
:10069600EB9FF5F0EA9E42F0E99D42F0EC6480C8DB
:0606A60064809845F0227B
:1006AC00EB9FF5F0EA9E42F0E99D42F0E89C45F0A4
:0106BC00221B
:1006BD00E86010ECA2E713FCED13FDEE13FEEF1353
:0406CD00FFD8F02240
:0C06D100E6FC08E6FD08E6FE08E6FF2255
:0D06DD00E6FB08E6F908E6FA08E6CBF8228D
:0C06EA00ECF608EDF608EEF608EFF6223C
:1006F600D083D082E493F608740193F608740293CB
:09070600F608740393F674047301
:10070F00D083D082F8E4937012740193700DA3A379
:10071F0093F8740193F5828883E47374029368608D
:06072F00EFA3A3A380DF8D
:00000001FF
